:100000000C9470010C948F010C948F010C948F014F
:100010000C948F010C948F010C948F010C948F0120
:100020000C948F010C948F010C94B7060C948F01E3
:100030000C948F010C948F010C948F010C948F0100
:100040000C948F010C948F010C948F010C948F01F0
:100050000C948F010C948F010C948F010C948F01E0
:100060000C948F010C948F010C948F010C948F01D0
:100070000C948F010C948F010C948F010C948F01C0
:100080000C948F010C948F010C948F010C948F01B0
:100090000C948F010C948F01002C2AE1080C11069E
:1000A0001712160915101A14040B071C0F13050D4F
:1000B000180A191B0E1D002B363733342F303138F8
:1000C0001E1F20212223242526272D2E2835E2E05D
:1000D000504F52514B4E494C4A4D4648E539E3E7A3
:1000E0003A3B3C3D3E3F40414243444529290000C4
:1000F00000000151000002520000044F00000551B1
:100100004F0006524F0008500000095150000A529B
:1001100050000C3800000D5138000E5238001437D2
:1001200000001551370016523700183600001951DB
:1001300036001A523600200B0000210B5100220B12
:100140005200240B4F00280B5000340B3700380BA3
:100150003600401D000041511D0042520600444F30
:100160001D0048501D004C1D380050060000515124
:10017000060052524D00544F0600585006005C06CF
:100180003800600B510062521D00700B06008004A5
:1001900000008151040082520400844F0400885002
:1001A00004008C04380091512C0092522C00944F82
:1001B0002C0098502C009C382C00A00B0400B00B95
:1001C0003800C04D0000C1514D00C44F4D00C85013
:1001D0004D00CC384D00D4374D00D8364D00E00BE3
:1001E0004D0012010002000000400000020000105B
:1001F0000102030109023B00020100C032090400B0
:10020000000103000200092101100001223400074F
:10021000058103080005090401000103000101092B
:100220002101100001223B00070582030800050C94
:10023000034F0054004C004C004300260343006869
:10024000006F007200640069007400650020007097
:100250000072006F0074006F007400790070006518
:10026000000C0330002E0030002E00310004030982
:100270000405010902A1010901A1000509190129CB
:10028000031500250175019503810275059501810E
:100290000105010930093109381581257F75089557
:1002A000038106C0C005010906A101050719E0295F
:1002B000E7150025017501950881028101190029C2
:1002C0006515002565750895068100050819012941
:1002D000051500250175019505910295039101C051
:1002E00011241FBECFEFD0E2DEBFCDBF11E0A0E0F2
:1002F000B1E0ECE5F4E100E00BBF02C007900D9225
:10030000A430B107D9F711E0A4E0B1E001C01D921B
:10031000A432B107E1F70E9408060C942D0A0C9450
:100320000000833039F5613069F0613028F06230C7
:1003300079F06330F9F412C084E0809320018DE6F7
:1003400092E011C08CE0809320018FE292E00BC01C
:1003500086E2809320018BE392E005C08CE08093DD
:10036000200181E692E0909322018093210181E0B7
:1003700090E0089580E090E00895CF93DF93CDB7AB
:10038000DEB722970FB6F894DEBF0FBECDBF8091C7
:10039000F10080931D018091F10080931E018091F6
:1003A0001D0190911E01009719F0019781F406C07C
:1003B00084E38093200181E792E005C08BE3809382
:1003C000200185EA92E0909322018093210180919F
:1003D000F10089838091F1008A838091E800877F12
:1003E0008093E80029813A818091200190E0821772
:1003F000930770F48F739070892B11F441E001C062
:1004000040E0E0912101F0912201909120011AC079
:1004100020932001F5CF8091E80080FFFCCF30E0F1
:100420000AC03F5F292F2150313439F084918093E5
:10043000F1003196922F9923A1F78091E8008E7FE9
:100440008093E800992359F08091E80082FFE3CF80
:10045000F0932201E09321019093200106C0F093D4
:100460002201E0932101109220018091E8008E7F0B
:100470008093E8008091E80082FD0BC0413029F4B0
:100480008091E8008E7F8093E8008091E80082FFF1
:10049000FCCF8091E8008B7F8093E8008091E8009A
:1004A0008F778093E80022960FB6F894DEBF0FBED8
:1004B000CDBFDF91CF9108958091E800877F809331
:1004C000E8008091E8008E7F8093E8008091E8004A
:1004D00082FFFCCF8091E8008B7F8093E8008091C1
:1004E000E8008F778093E8008091E8008E7F80930A
:1004F000E80008958091F1008091F1008091F10071
:1005000080931D018091F10080931E018091E8008D
:10051000877F8093E8008091E8008E7F8093E800D9
:100520008091E80080FFFCCF08958091F1008091D8
:10053000F1008091F10080931D018091F100809382
:100540001E018091E800877F8093E8008091E80099
:100550008E7F8093E8008091E80080FFFCCF0895B3
:10056000CF93DF93CDB7DEB722970FB6F894DEBFF7
:100570000FBECDBF8091F10080931D018091F100ED
:1005800080931E0180911D0190911E01009719F02A
:10059000019781F406C089E08093200186E092E013
:1005A00005C089E0809320018FE192E090932201C1
:1005B000809321018091F10089838091F1008A83E9
:1005C0008091E800877F8093E80029813A818091BB
:1005D000200190E08217930770F48F739070892B3D
:1005E00011F441E001C040E0E0912101F0912201CD
:1005F000909120011AC020932001F5CF8091E8004E
:1006000080FFFCCF30E00AC03F5F292F21503134FA
:1006100039F084918093F1003196922F9923A1F7BC
:100620008091E8008E7F8093E800992359F08091B3
:10063000E80082FFE3CFF0932201E0932101909341
:10064000200106C0F0932201E093210110922001C5
:100650008091E8008E7F8093E8008091E80082FD21
:100660000BC0413029F48091E8008E7F8093E80030
:100670008091E80082FFFCCF8091E8008B7F80931F
:10068000E8008091E8008F778093E80022960FB60B
:10069000F894DEBF0FBECDBFDF91CF91089580915A
:1006A000F1008091F100693071F06A3089F06630B4
:1006B000A1F4813229F0823281F40E94BD010AC086
:1006C0000E94B00207C0823041F40E945C0202C066
:1006D0000E94950281E090E0089580E090E0089506
:1006E0000F931F9309EE10E081E0F801808360E032
:1006F00081EC0E943F0682E0F801808360E081EC9B
:100700000E943F061F910F910895109214011092BC
:100710001501109216011092170110921A01E2EEC3
:10072000F0E0808184608083089580911A018F5F5A
:1007300080931A010895E0EEF0E08081816080836B
:10074000089580911A01833008F487C010921A012D
:1007500010921401109215011092160110921701B7
:100760000E945F04482F882329F480910501882383
:1007700021F473C08E3109F470C0642F70E09B01C6
:100780002F7030702A30310531F48091160181507C
:100790008093160125C02230310559F4809116014D
:1007A000815080931601809115018F5F8093150110
:1007B00020C02330310531F4809115018F5F809383
:1007C00015011EC02130310559F4809116018F5F4B
:1007D00080931601809115018F5F8093150113C0DE
:1007E0002530310531F4809116018F5F8093160119
:1007F00017C02430310521F4809116018F5F09C0A4
:100800002C30310541F02830310551F4809116012A
:1008100081508093160180911501815080931501BC
:10082000CB01807390708031910521F48091140187
:1008300081600CC08032910521F4809114018260A6
:1008400005C0C09729F4809114018460809314013D
:100850004093050181E090E0089580E090E00895E4
:100860001F9310910601113041F580911F018823DB
:1008700021F10E94A103882301F11093E9008091E6
:10088000E80085FF1AC0809114018093F1008091E7
:1008900015018093F100809116018093F100809101
:1008A00017018093F1008091E8008E7F8093E8002B
:1008B0008091E8008F778093E8001F910895CF938F
:1008C000DF93CDB7DEB724970FB6F894DEBF0FBE27
:1008D000CDBF83B18095898383B180958A8383B1AD
:1008E00080958B8383B180958C8320E030E0BE01BE
:1008F0006F5F7F4F09C083B19370FB01E90FF11D5A
:10090000809580832F5F3F4F922F49818A814817BE
:1009100091F78B81481779F78C81481761F74093DD
:100920000C01442329F480910B01882379F565C0DB
:100930004E3161F580910B018E3141F180910601BC
:100940008F5F80930601833010F0109206015C984F
:100950005F9880910601813061F0813018F082301B
:10096000A9F40FC084E690E0909301018093000108
:100970000DC084E690E090930101809300015C9AA1
:1009800005C010920101109200015F9A90910B0135
:10099000242F2923291771F010920A0110920901BE
:1009A00040930B0180910201882339F110920201DA
:1009B000892F21C0822F842B821751F081E08093F0
:1009C000020110920A011092090140930B0115C017
:1009D0002091090130910A0180910001909101015B
:1009E0002817390738F42F5F3F4F30930A012093BF
:1009F000090103C0842F90E002C080E090E02496BB
:100A00000FB6F894DEBF0FBECDBFDF91CF91089532
:100A100014B88FEF85B98AB1806F8AB910921A0124
:100A2000E2EEF0E08081846080830895282F88239F
:100A300069F480910701803EF0F58823E1F110927E
:100A400007011092080180E090E00895833EF1F0E4
:100A5000843E38F4813E91F0823EA0F4803E59F508
:100A600009C0853ED9F0853EA8F0863ED9F0873E84
:100A700011F51CC08091080181601BC080910801A4
:100A8000826017C080910801846013C080910801C2
:100A900088600FC08091080180610BC080910801BF
:100AA000806207C080910801806403C080910801C2
:100AB00080688093080190910801992311F05D9A54
:100AC00001C05D98293329F480910701893309F029
:100AD0004E9A20930701892F90E008951F93182FB5
:100AE0004CE330E0642F630F712D711DCB0162E088
:100AF00070E00E94060A862F90E0FC01EE0FFF1FB7
:100B0000EE0FFF1FE251FF4F2491121718F4462FEA
:100B1000415004C0211730F4362F3F5F431710F7C0
:100B200080E090E01F9108951F938091060181302D
:100B300009F46CC082E08093E9008091E80080FFB6
:100B400065C080911F01882309F460C08091E8008E
:100B500080FFFCCF0E945F0480931C01109106016E
:100B6000112321F0123009F051C01FC0863510F05A
:100B700010921C01E0911C01F0E0E856FF4FE49157
:100B8000E0931C0182E08093E9008E2F0E941605FD
:100B90008093F1001092F10080911C018093F1008C
:100BA0001092F1001092F10021C00E946E05809316
:100BB0001C011093E9001092F1001092F10090E0F6
:100BC000880F991F880F991FFC01E151FF4FE49195
:100BD000E093F100FC01E051FF4FE491E093F1005C
:100BE0008F509F4FFC0184918093F1001092F1008F
:100BF0001092F1001092F1008091E8008E7F8093B6
:100C0000E8008091E8008F778093E8001F910895B5
:100C1000A89587EF84BFE0E6F0E08081886180835B
:100C20001082E1E6F0E080E8808310820E94010AF1
:100C300080E090E0089513BE83B7856083BF8895F8
:100C4000089513BE83B7816083BF8895089513BE4E
:100C500083B7836083BF8895089513BE83B7876089
:100C600083BF8895089513BE83B78D6083BF889531
:100C7000089513BE83B78F6083BF889508959091C0
:100C8000EB0091609093EB008093EC008091ED007D
:100C90008270862B8093ED008091ED0082608093BE
:100CA000ED008091EE00992787FD90958827990F98
:100CB000881F992708954091F40020E030E0822FAA
:100CC00040FF02C090E008952F5F3F4F273031056D
:100CD00011F04695F4CF80E090E00895FB018093F9
:100CE000E90004C081918093F10041508091E800B7
:100CF00085FF02C04423B1F7842F90E00895FB01E3
:100D00008093E90004C08091F1008193415080916B
:100D1000E80085FF02C04423B1F7842F90E00895D6
:100D20008093E900EBEEF0E080818062808308959B
:100D30008091D8008F7B8093D8008091D90081FF6B
:100D40000EC01092E9008091EB0080FD08C0109267
:100D5000E90060E382E00E943F0690E0089580E0B1
:100D600090E00895089578940E941B0608951F92BC
:100D70000F920FB60F9211242F933F934F935F93CF
:100D80006F937F938F939F93AF93BF93EF93FF9353
:100D90008091DA0080FF33C08091D80080FF2FC09F
:100DA0008EEF8093DA008091D90080FF19C081E036
:100DB0008093230180910D0190910E0182609093A8
:100DC0000E0180930D018091E20088608093E20023
:100DD0000E94AA098091E0008E7F8093E0000FC0FE
:100DE0000E949B031092230110921F0180910D011C
:100DF00090910E01846090930E0180930D0180917B
:100E0000E10082FF09C08091E20082FF05C08BEF04
:100E10008093E1000E9495038091E10080FF1FC054
:100E20008091E20080FF1BC08EEF8093E1008091F3
:100E3000E20080618093E2008FEE8093E100809178
:100E4000D80080628093D80080910D0190910E01AE
:100E5000806290930E0180930D010E94B3068091F1
:100E6000E10084FF1AC08091E20084FF16C08091E7
:100E7000D8008F7D8093D8008FEE8093E100809121
:100E8000E2008F7E8093E20080910D0190910E012F
:100E9000806490930E0180930D018091E10085FFA5
:100EA0001AC08091E20085FF16C08091E2008F7E1B
:100EB0008093E2008FED8093E1008091E2008F7DCE
:100EC0008093E20080910D0190910E0180689093D3
:100ED0000E0180930D018091E10083FF12C080918B
:100EE000E20083FF0EC087EF8093E1000E94980626
:100EF00080910D0190910E01916090930E0180936D
:100F00000D01FF91EF91BF91AF919F918F917F91D3
:100F10006F915F914F913F912F910F900FBE0F9066
:100F20001F9018950E94C6090895E7EDF0E08081B2
:100F30008160808380818F7B8083808180688083D3
:100F40000E9499090895CF93DF93CDB7DEB722971A
:100F50000FB6F894DEBF0FBECDBF9091F100909315
:100F600013016091F1006630F9F0673068F4613088
:100F700009F400C1613008F46AC1633009F433C177
:100F8000653009F0BEC1BCC0693009F4DAC06A300E
:100F900020F4683009F0B5C197C06A3009F499C1EE
:100FA0006B3009F0AEC19CC1903809F08BC0109233
:100FB0000F016091F1008091F100813019F08230D1
:100FC00089F406C082E18093200182EE91E005C0A1
:100FD0008BE38093200184EF91E090932201809332
:100FE000210105C00E949101882309F48FC18091DD
:100FF000F1008091F1008091F10089838091F100EE
:101000008A838091E800877F8093E80029813A8174
:101010008091200190E08217930758F48F739070AD
:10102000892B21F481E080930F0105C010920F01FC
:1010300002C020932001E0912101F09122019091C2
:10104000200117C08091E80080FFFCCF30E00AC08B
:101050003F5F292F2150313439F084918093F10082
:101060003196922F9923A1F78091E8008E7F80938B
:10107000E800992359F08091E80082FFE3CFF093D4
:101080002201E09321019093200106C0F0932201F8
:10109000E0932101109220018091E80082FD10C1AF
:1010A00080910F01813049F48091E80080FFFCCFEE
:1010B0008091E8008E7F8093E8008091E80082FFB5
:1010C000FCCFFEC066E008C19038C1F48091E80012
:1010D000877F8093E80080911F018093F1008091C9
:1010E000E8008E7F8093E8008091E8008F778093FE
:1010F000E8008091E80082FFFCCFE2C068E0ECC02D
:101100009923E9F49091E3008091F1008F77907832
:10111000892B8093E3008091E800877F8093E8002B
:101120008091E8008E7F8093E8008091E80080FF46
:10113000FCCF8091E30080688093E300F1C065E01C
:10114000CBC09923A9F49091F100923008F0DEC051
:101150008091E800877F8093E80090931F01809141
:10116000E8008E7F8093E800892F0E947003D8C02A
:1011700069E0B2C09330A8F5992309F4C7C0913053
:1011800009F4C4C08091F1009091F100882309F026
:10119000BDC0E091F100EF77E093E9008091EB00B2
:1011A00080FF50C0EE23B1F08091EB00806180930E
:1011B000EB0081E090E00E2E02C0880F991F0A9488
:1011C000E2F78093EA001092EA008091EB008860D9
:1011D0008093EB001092E900F0E0E05FFE4F108298
:1011E00028C061E079C0933080F5913009F48EC059
:1011F000923009F095C08091F1009091F100882320
:1012000009F084C0E091F100EF7709F47FC0E0932A
:10121000E9008091EB0080FF15C08091EB008062B7
:101220008093EB001092E900F0E0E05FFE4F81E078
:1012300080838091E800877F8093E8008091E800B8
:101240008E7F6CC01092E90061C063E045C0892FB9
:101250008058833008F040C08091F1008091F10007
:10126000E091F100913861F0923891F0903809F0F6
:101270004DC08091E800877F8093E80081E013C033
:101280008091E800877F8093E8001092F1000DC004
:101290008091E800877F8093E800F0E0EF77F070BE
:1012A000E05FFE4F80818093F1001092F100809109
:1012B000E8008E7F8093E8008091E80082FFFCCFF9
:1012C0008091E8008B7F8093E8008091E8008F7721
:1012D00025C09138D9F06AE0892F0E944F0320C0C1
:1012E0009130F1F48091E800877F8093E80080914D
:1012F000E8008E7F8093E8008091E80080FD10C0B8
:10130000FBCF892F0E944F03882351F48091EB007B
:1013100080628093EB008091E800877F8093E800F3
:1013200022960FB6F894DEBF0FBECDBFDF91CF91EE
:1013300008957894E8EDF0E080818F768083808155
:101340008069808380818F7B8083808181608083BE
:10135000789408958EE089BD09B400FEFDCF809198
:10136000D8008F7D8093D8008091E20081608093C7
:10137000E2008091E20088608093E2000E9498067B
:101380008091E0008E7F8093E00008958091D900E5
:1013900080FF09C080912301882329F481E0809394
:1013A00023010E94AA0980910D0190910E0190FFE6
:1013B00010C080910D0190910E019E7F90930E01BF
:1013C00080930D0181E08093EA001092EA00109270
:1013D0001F011092E9008091E80083FF02C00E9483
:1013E000A307089508950E9492070E9430040E9466
:1013F0009405F9CF0E9495070E9485030E94080575
:1014000008950E94FA090E94F309089597FB092E96
:1014100007260AD077FD04D00CD006D000201AF49D
:10142000709561957F4F0895F6F7909581959F4F40
:101430000895AA1BBB1B51E107C0AA1FBB1FA6171B
:10144000B70710F0A61BB70B881F991F5A95A9F76D
:0C14500080959095BC01CD010895FFCF60
:04145C006400010027
:00000001FF
